:02000000E52EEB
:100DCA00F701F801F901FA01FB018301272F4030ED
:100DDA0083168F00831285010B308316850031300C
:100DEA009F000730831299000800F40080308312B4
:100DFA009F007408F20002300310F20DFF3E031D3B
:100E0A00012F1F0872079F001F140B2F0C2F64005D
:100E1A0083120C139F14112F9F18142F152F112FA3
:100E2A00162F1E08F200F3017208F300F20183166E
:100E3A001E087207F0000030031801307307F10032
:100E4A00262F0800EC268312051205114130F60000
:100E5A00EE30F500F50B2F2FF60B2F2F6400F9015A
:100E6A00362F0130F5007508F9071030F500F50B3B
:100E7A003C2F6400C9307902031C442F452F362FBA
:100E8A00F9010030FA267108F801F8077008F7012D
:100E9A00F7077808F6007708F50002300310F60C19
:100EAA00F50CFF3E031D532F7508F7007608F8006E
:100EBA007708F5007508FB00E1307B02031C662FFA
:100ECA00672F6E2F0530F5007508FA008312051694
:100EDA00F12FC1307B02031C732F742F7B2F063036
:100EEA00F5007508FA0083120516F12FB1307B025E
:100EFA00031C802F812F882F0730F5007508FA0010
:100F0A0083120516F12FA1307B02031C8D2F8E2F21
:100F1A00952F0830F5007508FA0083120516F12F8F
:100F2A0091307B02031C9A2F9B2FA22F0930F500C8
:100F3A007508FA0083120516F12F81307B02031C13
:100F4A00A72FA82FAF2F0A30F5007508FA008312D1
:100F5A000516F12F71307B02031CB42FB52FBC2F5D
:100F6A000C30F5007508FA0083120516F12F61306E
:100F7A007B02031CC12FC22FC92F0E30F500750842
:100F8A00FA0083120516F12F51307B02031CCE2F73
:100F9A00CF2FD62F1130F5007508FA0083120516E7
:100FAA00F12F41307B02031CDB2FDC2FE32F1330A0
:100FBA00F5007508FA0083120516F12FFB01FA01F4
:100FCA0083120512F12FF12FF12FF12FF12FF12FAB
:100FDA00F12FF12FF12FF12F7B0883169200831244
:100FEA009101053092000C3095007A089300362F53
:060FFA00362F362F0028FF
:084000000000070001000000B0
:02400E00C4F3F9
:00000001FF
